:100000000C942D000C943F000C943F000C943F0086
:100010000C943F000C943F000C943F000C943F0064
:100020000C943F000C943F000C943F000C943F0054
:100030000C943F000C943F000C943F000C943F0044
:100040000C943F000C943F000C94F4000C943F007F
:100050000C943F006D63312E300011241FBECFE59C
:10006000D8E0DEBFCDBF24E0A0E6B0E001C01D9225
:10007000AC36B207E1F70E9434010C941B020C94D9
:10008000000083E088BB80E182BB82BB94E192BB2D
:1000900092BB82BB82BB92BB21E028BB82BB82BBEE
:1000A00092BB28BB82BB82BB92BB28BB82BB82BBFC
:1000B00092BB82BB82E08EBD1DBC1CBC8CB5853062
:1000C000E8F394E192BB92BB80E182BB82BB92BB1E
:1000D00092BB82BB82BB92BB26B321702093640487
:1000E00082BB82BB92BB26B330916404330F217074
:1000F000232B2093640482BB82BB92BB26B3309136
:100100006404330F2170232B2093640482BB82BBD1
:1001100092BB26B330916404330F2170232B2093BC
:10012000640482BB82BB92BB26B32170209365041A
:1001300082BB82BB92BB26B330916504330F217022
:10014000232B2093650482BB82BB92BB26B33091E4
:100150006504330F2170232B2093650482BB82BB7F
:1001600092BB26B330916504330F2170232B20936B
:10017000650482BB82BB92BB26B330916504330F0A
:100180002170232B2093650482BB82BB92BB26B3D4
:1001900030916504330F2170232B2093650482BBBB
:1001A00082BB92BB26B330916504330F2170232BA1
:1001B0002093650482BB82BB92BB86B39091650499
:1001C000990F8170892B809365048CE182BB8091AB
:1001D000640490E0982F882720916504822B9093E7
:1001E00067048093660408951F920F920FB60F92D2
:1001F00011242F933F934F935F936F937F938F932C
:100200009F93AF93BF93EF93FF930E944100E091C0
:100210006604F0916704F695E795F695E795F695EF
:10022000E795F0936704E0936604EE0FFF1FEC5927
:10023000FF4F8081918101969183808381E080933B
:100240006000AF98AF9AFF91EF91BF91AF919F91EE
:100250008F917F916F915F914F913F912F910F906F
:100260000FBE0F901F90189582E087BB9CE991BB51
:1002700090E894BB95BB98E19AB910BC9CE099B901
:1002800096EA90BD90E498B98EBD109269041092E0
:10029000680488E2E82E94E4F92EC1E0D0E02BE473
:1002A000A22E33E4B32E43E0C42E44E0D42E02E069
:1002B00014E080916804909169045F9BFECFFC017B
:1002C000019690936904809368042CB1EE59FF4F16
:1002D0002083E89EA001E99E500D11242091620028
:1002E00030E02417350748F7109261001DBC1CBC94
:1002F00080916200F0926200D0936904C093680418
:100300008A3009F470C0B8F08C3009F45EC008F48B
:1003100056C08D3009F04FC04398809162005D9BBC
:10032000FECF8CB980916200843409F11092690487
:1003300010926804BECF813009F460C08230D9F5D4
:100340000E9441008091680490916904FC01EE597B
:10035000FF4F209165042083029690936904809357
:10036000680480916404818380916200D8CFD09327
:100370006B04C0936A0480916804909169040297A9
:10038000A8F281E090E05D9BFECFFC01EE59FF4FAB
:1003900080818CB980916A0490916B04019690934E
:1003A0006B0480936A042091680430916904821779
:1003B000930748F3BBCFB092620083E4B0CF1093B1
:1003C00069040093680484E4AACFE3E6F0E01192A4
:1003D00084E0E536F807D9F7D0926B04C0926A043E
:1003E000809162009CCFBB9880B7877F80BFA8B800
:1003F000AF98AF9A78948091620091CF45E050E039
:1004000064E570E083E690E00E9412028091680447
:100410009091690405969093690480936804809193
:1004200062007DCFFB01DC0102C005900D924150BE
:0A0430005040D8F70895F894FFCF6C
:00000001FF
